:1000000063C000007DC000007BC0000079C000001C
:1000100077C0000075C0000073C0000071C0000010
:100020006FC000006DC000000C94550969C000004D
:1000300067C0000065C0000063C0000061C0000030
:100040005FC000005DC000005BC0000059C0000040
:1000500057C0000055C00000B6C40000510A802AF5
:100060000000000A00FF000059551801111E111B65
:10007000500B411B411F1101511F511B000000007B
:1000800000000000000000000000510F91394114F1
:100090009131411E410E411D500F802010154886A0
:1000A0004014780570855115510E5195518E21904F
:1000B00081205015484450C528C028200950000010
:1000C000000000000000000011241FBECFEFD4E0AC
:1000D000DEBFCDBF11E0A0E0B1E0ECEAF9E102C083
:1000E00005900D92AA38B107D9F712E0AAE8B1E05D
:1000F00001C01D92AB30B107E1F79DD00C94D40C38
:100100007FCF06C020E000002F5F2D37E1F7019779
:100110000097C1F7089580E88093610083E08093A1
:1001200061001092700088E08093B60088EC8093A4
:10013000B30010926E0081E0809381008093B00044
:100140002091B6008091B60090E08470907030E00D
:1001500021703070822B932B892B91F788EE93E0DE
:10016000D0DF3FEF41E0F89436BB37BB10928500FB
:10017000109284001092B200B99BFECF10928100C1
:100180007894B09916C0209184008091850090E009
:10019000982F8827820F911D28E18B36920724F033
:1001A00080916600815008C0885E974114F081E01C
:1001B00006C0809166008F5F8093660080E0409368
:1001C0008100882381F20895A6DFE1E6F0E080E86F
:1001D000808383E080830E944C098CE090E00E9441
:1001E0007E09D7D385B7806885BF85B7806885BF0E
:1001F00081E090E0909391018093900190938F0122
:1002000080938E018FEF9FEFAFEFBFEF809392014E
:1002100090939301A0939401B0939501109296014D
:1002200010929701109298011092990110929B01DF
:1002300010929A010895C8DF789480E091E073D419
:1002400000D086E091E0EDB7FEB7928381830E94F3
:10025000A7090F900F9088EE93E053DF6ED5FECF85
:100260002F923F924F925F926F927F928F929F92C6
:10027000AF92BF92CF92DF92EF92FF920F931F93B4
:10028000DF93CF9300D000D00F92CDB7DEB78B8332
:1002900080937C00813051F480917C00806C80934D
:1002A0007C002B99FECF2B9BFECF0AC080917C0057
:1002B000806480937C0080917C008F7780937C00A9
:1002C00083E880937A0080917A00806480937A003A
:1002D00080917A0084FFFCCF2091900130919101B0
:1002E0003A8329831D821C820F2EF0E02F2EF0E02E
:1002F0003F2EF0E04F2EF0E05F2EF02D4201310155
:1003000057C080917A00806480937A0080917A004F
:1003100084FFFCCF6091780070E080E090E00E9464
:10032000DB0A7B018C016091790070E0762F6627F3
:10033000882777FD8095982F0E94DD0A9B01AC01EC
:10034000C801B7010E94DA097B018C01A201910169
:100350000E94D9095B016C018C819D8101969D836E
:100360008C83BC0180E090E00E94DB0A9B01AC0121
:10037000C601B5010E94420A9B01AC01C201B10154
:100380000E94DA091B012C01C801B701A2019101E9
:100390000E94D9099B01AC01C601B5010E948D0BD9
:1003A0009B01AC01C401B3010E94DA093B014C017D
:1003B000EC81FD8129813A81E217F30708F4A1CF8E
:1003C00080917A008F7780937A003B81032F10E031
:1003D000F801EE0FFF1FEE0FFF1FE257FE4F2686BC
:1003E0003786408A518AC401B30120E030E040E002
:1003F00050E00E943E0A882324F497FA909497F8DC
:100400009094000F111F000F111F02571E4FE9811A
:10041000FA81BF0180E090E00E94DB0A9B01AC0101
:10042000C401B3010E94420AF80166A777A780AB16
:1004300091ABC201B1010F900F900F900F900F90F0
:10044000CF91DF911F910F91FF90EF90DF90CF90B0
:10045000BF90AF909F908F907F906F905F904F90E4
:100460003F902F900895B0DE80E00895FC018081D8
:10047000882339F0CF010E94AF0C90938F018093B5
:100480008E0100D000D082E191E0EDB7FEB79283FB
:10049000818380918E0190918F019483838357D7BC
:1004A0008FE191E0EDB7FEB79283818380918E0159
:1004B00090918F019483838316D40F900F900F90A7
:1004C0000F9080E00895FC018081882379F0CF01AE
:1004D0000E94AF0CAA2797FDA095BA2F8093920196
:1004E00090939301A0939401B093950100D000D014
:1004F00000D088E291E0EDB7FEB7928381838091CE
:10050000920190919301A0919401B0919501838300
:100510009483A583B6831BD787E391E0EDB7FEB73D
:10052000928381838091920190919301A091940193
:10053000B091950183839483A583B683D4D38DB77B
:100540009EB706960FB6F8949EBF0FBE8DBF80E093
:100550000895FC018081882339F0CF010E94AF0CFF
:10056000909391018093900100D000D082E491E0BB
:10057000EDB7FEB7928381838091900190919101B4
:1005800094838383E4D68EE491E0EDB7FEB7928343
:100590008183809190019091910194838383A3D36F
:1005A0000F900F900F900F9080E00895FC018081D4
:1005B000882341F0CF010E94AF0C90939B01809360
:1005C0009A0144D100D000D086E591E0EDB7FEB7A6
:1005D0009283818380919A0190919B01948383837C
:1005E000B6D681E691E0EDB7FEB792838183809124
:1005F0009A0190919B019483838375D30F900F9000
:100600000F900F9080E00895AF92BF92CF92DF924B
:10061000EF92FF920F931F93CF93DF936C01DC0156
:100620008C91882331F0E6012AE6A22E21E0B22E39
:1006300056C000E0C6E6D1E0802F12DE00D000D028
:1006400000D0EDB7FEB7D283C183ADB7BEB7139666
:100650006D937D938D939C93169779D60F5FEDB72D
:10066000FEB736960FB6F894FEBF0FBEEDBF08304A
:1006700019F75CC08053F4DD7B018C01E991F0E057
:10068000EE0FFF1FEE0FFF1FE253FF4F66A577A58A
:1006900080A991A90E94F40B2DB73EB72A50304093
:1006A0000FB6F8943EBF0FBE2DBFEDB7FEB7319623
:1006B000ADB7BEB71296BC92AE921197E282F382AA
:1006C00004831583668377838087918740D6EDB74F
:1006D000FEB73A960FB6F894FEBF0FBEEDBF888105
:1006E000882341F600D000D00DB71EB70F5F1F4F13
:1006F00081E791E0ADB7BEB712969C938E931197A8
:10070000D601EC91F0E0EE0FFF1FEE0FFF1FE2535A
:10071000FF4F668577858089918921D7F80173839A
:100720006283E1D20F900F900F900F9000D084E77A
:1007300091E0ADB7BEB712969C938E93119707D6F2
:100740000F900F9080E0DF91CF911F910F91FF905C
:10075000EF90DF90CF90BF90AF900895CF92DF924F
:10076000EF92FF920F931F93CF93DF93EC0187E7F4
:1007700091E0D9D1EE24FF2487013CE7C32E31E07C
:10078000D32E109296011092970110929801109218
:10079000990100D000D000D0EDB7FEB7D282C1825F
:1007A000E382F48205831683D2D58DB79EB7069671
:1007B0000FB6F8949EBF0FBE8DBFCE0125DF888196
:1007C000882319F08981843749F481E0DCD1C8019C
:1007D000B701F0D103C0B2D5882329F52091960145
:1007E00030919701409198015091990180918E012B
:1007F00090918F01A0E0B0E0281739074A075B0706
:1008000050F3E20EF31E041F151F80919201909188
:100810009301A0919401B0919501E816F9060A0799
:100820001B0708F4AECF80E0AED180E0DF91CF911E
:100830001F910F91FF90EF90DF90CF9008958FEB75
:1008400084B98FEF85B986E585B90895CF93DF9395
:10085000EC01F5DF2B99FECF85B1866085B92B9B26
:10086000FECF2B99FECF299828982B9BFECF2B9952
:10087000FECF289A2B9BFECF2B99FECF80E1C03074
:10088000D80724F02898D595C79501C0289A2B9BA6
:10089000FECF2B99FECF289A2B9BFECF2B99FECF14
:1008A0002BE030E0CE01022E02C0959587950A9488
:1008B000E2F780FD02C0289801C0289A2B9BFECF4A
:1008C0002B99FECF215030408FEF2F3F380751F743
:1008D000299A2B9BFECF2B99FECF2A982B9BFECFDC
:1008E0002B99FECF2A9A2B9BFECF2B99FECFDF911F
:1008F000CF910895CF93DF93982F6630C8F58A5231
:10090000813518F0A0E0B0E00CC0913608F09F7D72
:100910009A52E92FF0E0EE0FFF1FE45AFF4FA59126
:10092000B491862F90E0EC01C170D07060FD02C0E0
:1009300090EF01C09FE0669570E063527E4F20E02B
:1009400030E0FB01E20FF31F4A2F4F7084E0B695B1
:10095000A7958A95E1F7209711F04295407F808115
:100960008923482B40832B5F3F4F2431310549F7C2
:10097000DF91CF91089581118FEF20E030E0F901F0
:10098000E352FE4F80832F5F3F4F24313105B9F78B
:10099000089580E0F0DFA7EEB0E08C918F608C933B
:1009A00087EB8093E50087E08093E600E4EEF0E0DB
:1009B00080EC80838081886080838C91806E8C93B2
:1009C00010928A0108951F920F920FB60F92112470
:1009D000EF92FF920F931F932F933F934F935F9349
:1009E0006F937F938F939F93AF93BF93CF93DF9337
:1009F000EF93FF9300918901015000938901809149
:100A0000DC01882381F0002381F480918B0188230D
:100A100021F481E080938A0108C080918B0181508C
:100A200080938B0102C010920A0280918A0181306A
:100A300009F051C0E0908C01FF2410E0C0E0D0E04C
:100A40006C2F80910A02992787FD90958C0F9D1F2E
:100A500097FD15C0112399F4E0910A02FF27E7FDE5
:100A6000F095EC0FFD1FEF50FE4F8081F82EFF1C1C
:100A7000FF24FF1C8F7721F41C2F1F5F01C080E231
:100A8000FF2021F094E09E1508F480E233DF2196E8
:100A9000C630D105A9F6ACEEB0E0FD01EF50FF4F36
:100AA00080818D9381E0A030B807B9F780918D01E6
:100AB000882321F081E08093F40002C01092F400BA
:100AC000113011F48AEF03C080910A028F5F809386
:100AD0000A0210928A01002319F483E080938901AD
:100AE00080918C018A3019F410928C0105C080919C
:100AF0008C018F5F80938C01FF91EF91DF91CF91FB
:100B0000BF91AF919F918F917F916F915F914F9125
:100B10003F912F911F910F91FF90EF900F900FBE7B
:100B20000F901F901895BC0180918A018823E1F7EE
:100B300020E030E006C0F901EF50FE4F80832F5FC8
:100B40003F4F422FFB01E20FF31F8081882319F0F2
:100B50002931310581F7E42FF0E0EF50FE4F10828C
:100B6000473048F081E08093DC0110920A0283E074
:100B700080938B0104C01092DC0110920A0281E084
:100B800080938A01089580938D010895982F809114
:100B90008A018823E1F76093DC0110920A029093A6
:100BA0008A010895893128F4E82FF0E0EF50FE4FD4
:100BB000608308956F927F928F929F92AF92BF92BF
:100BC000CF92DF92EF92FF920F931F93DF93CF9319
:100BD00000D000D000D0CDB7DEB75B016C0120E4BF
:100BE0003EE745E050E099D639014A01B90180E07D
:100BF00090E020EC31E84AEF5FEF49D67B018C01B1
:100C0000EA0CFB1C0C1D1D1DC801B70120E737E1D4
:100C100040E050E082D659016A0180E797E19C01EB
:100C20002A9DC0012B9D900D3A9D900D1124A0E0AE
:100C3000B0E0E81AF90A0A0B1B0BC801B70124E659
:100C400030E040E050E069D689019A01C3016AE0D2
:100C500070E03CD66983C3016AE070E037D68A83CE
:100C6000C5016AE070E032D66B83C5016AE070E0CE
:100C70002DD68C83C8016AE070E028D66D83C80148
:100C80006AE070E023D68E837E010894E11CF11C9B
:100C9000870187E0C82ED12CCC0EDD1E802F8E1947
:100CA000F80161918F01605D7DDF0C151D05B1F7C5
:100CB00086E060E077DF81E060E068DF26960FB6CF
:100CC000F894DEBF0FBECDBFCF91DF911F910F9182
:100CD000FF90EF90DF90CF90BF90AF909F908F905C
:100CE0007F906F900895EF92FF920F931F93DF9381
:100CF000CF93CDB7DEB769970FB6F894DEBF0FBEBE
:100D0000CDBFFE01B296619171917E010894E11C04
:100D1000F11CC701AF013DD28C01C70104DFC8013E
:100D200069960FB6F894DEBF0FBECDBFCF91DF91AD
:100D30001F910F91FF90EF900895AF92BF92CF92C5
:100D4000DF92EF92FF920F931F93DF93CF93CDB774
:100D5000DEB72A970FB6F894DEBF0FBECDBF83E291
:100D6000DCD2E4D2D82ED9D2CC245E010894A11CC6
:100D7000B11CEC2CFF24DAD285010E0D1F1DD80109
:100D80008C93CBD2F80100810D3049F00E3018F46D
:100D90000A3049F404C0003239F00B3321F4EA0C74
:100DA000FB1CD7011C92C394EC2CFF24870101503B
:100DB0001040F501E00FF11F8081882319F0B9E0A0
:100DC000BC15B8F600D080E891E0EDB7FEB792838D
:100DD0008183BDD2FE0131960E0F1F1F0F900F9021
:100DE000D8018C91882369F083E891E09CDE00D0E3
:100DF00085E891E0EDB7FEB792838183A8D28FEFAB
:100E000047C0EE0DFF1D1082F4E6DF1611F1FD154F
:100E100050F081E2D81649F1A1E6DA1619F1BDE0E9
:100E2000DB1651F510C0E2E7DE1669F0ED1520F093
:100E3000F0E7DF1609F50AC084E7D81669F0A7E7DE
:100E4000DA16D1F40CC0E4E0F3E011C0EEEAF3E00E
:100E50000EC0E6EDF2E00BC0E3E6F2E008C0E6E328
:100E6000F2E005C0E9EAF2E002C0E3E3F2E0CE011D
:100E700001960995882371F083E891E054DE00D053
:100E800085E891E0EDB7FEB79283818360D28EEF63
:100E90000F900F902A960FB6F894DEBF0FBECDBF0D
:100EA000CF91DF911F910F91FF90EF90DF90CF9046
:100EB000BF90AF9008956F927F928F929F92AF9262
:100EC000BF92CF92DF92EF92FF920F931F93CF9337
:100ED000DF933C015A016B01411551056105710514
:100EE00019F080E090E01EC080E3F301808311825E
:100EF00041E050E03BC0C601B5012AE030E040E0EF
:100F000050E00BD57B018C01C601B5012AE030E031
:100F100040E050E002D559016A01F0E3EF0EF40120
:100F2000E082CE014301880E991EEC012196FAE081
:100F3000AF16B104C104D104F0F68A2D805DF4012E
:100F40008083AE01BE0175956795D30120E030E046
:100F500007C09C9180818D9390832F5F3F4F319785
:100F600026173707B4F3C60DD71D1882CA01DF91C3
:100F7000CF911F910F91FF90EF90DF90CF90BF9096
:100F8000AF909F908F907F906F900895EF92FF9217
:100F90000F931F93CF93DF937C01FB0161157105C4
:100FA00019F080E090E016C080E3D7018C93119691
:100FB0001C9241E050E02FC0CF016AE070E086D47F
:100FC0009C01CF016AE070E081D4FB01205DD80173
:100FD0002C93CE018701080F191FEC012196EA30EE
:100FE000F10550F78E2F805DF8018083AE01BE01C0
:100FF00075956795D70120E030E007C09C9180810E
:101000008D9390832F5F3F4F319726173707B4F3A7
:10101000CE0DDF1D1882CA01DF91CF911F910F9174
:10102000FF90EF900895CF92DF92EF92FF920F938F
:101030001F93CF93DF93EC018B016115710521F0B4
:10104000FB0180E090E014C080E38883198221E0F6
:1010500030E03BC0CF016AE070E04CD49C01CF018E
:101060006AE070E047D4FB01205DD7012C93C601F4
:101070007E01E80EF91E6C010894C11CD11CEA30F7
:10108000F10544F78E2F805DF7018083960117FFED
:1010900007C0FE01EC0DFD1D8DE280832F5F3F4FE9
:1010A000B90175956795FE01C20FD31FDE0140E0BF
:1010B00050E006C090818C9181939C934F5F5F4F6D
:1010C000119746175707B4F31882C901DF91CF91E2
:1010D0001F910F91FF90EF90DF90CF9008956F9246
:1010E0007F928F929F92AF92BF92CF92DF92EF92B8
:1010F000FF920F931F935C013A014B01CB01BA01A0
:1011000029D29B01AC017B01C501B9018CDF6C01C7
:10111000F501E80FF91F8EE280830894C11CD11CF1
:10112000AC0CBD1C0027F7FC0095102FC801B701BF
:1011300044D29B01AC01C401B3013BD120E030E0BB
:1011400048EC52E4EAD206D29B01AC01C501B901D8
:101150006ADF8C0D9D1D1F910F91FF90EF90DF9026
:10116000CF90BF90AF909F908F907F906F90089599
:101170009C0180E090E002C0EC930196FB01E80F37
:10118000F91FE081D901A80FB91FEE23A9F71C921E
:101190000895AF92BF92CF92DF92EF92FF920F939A
:1011A0001F93CF93DF937C015B01DA01C0E0D0E0B5
:1011B000CC24DD245AC0853209F04FC081818936A4
:1011C00091F08A3638F4843671F0863679F18336B8
:1011D00039F438C0833701F1853729F08C3669F04E
:1011E000CFEFDFEF4DC08D010E5F1F4F6D917C91F2
:1011F000C7018C0F9D1FCADE0BC08D010C5F1F4FF6
:101200004D915D916D917C91C7018C0F9D1F53DEB7
:10121000C80FD91FD8011DC08D010E5F1F4F6D91E2
:101220007C91C7018C0F9D1FA3DFF2CF8D010C5F56
:101230001F4F4D915D916D917C91C7018C0F9D1F4A
:101240004EDFE6CFF701EC0FFD1F8C9180832196D6
:1012500012960894C11CD11C05C0F701EC0FFD1FAC
:10126000808321960894C11CD11CF501EC0DFD1D55
:101270008081882309F09FCFEC0EFD1EF7011082BC
:10128000CE01DF91CF911F910F91FF90EF90DF90F2
:10129000CF90BF90AF900895239A82E080936E0024
:1012A00086E287BD8CE084BD08951F920F920FB631
:1012B0000F9211248F939F93AF93BF9380919601C8
:1012C00090919701A0919801B09199010196A11D6B
:1012D000B11D8093960190939701A0939801B093CC
:1012E000990185B198E0892785B9BF91AF919F9108
:1012F0008F910F900FBE0F901F901895292F3327B5
:101300002093C5008093C4001092C00088E18093B0
:10131000C10086E08093C2000895982F2E9A809194
:10132000C00085FFFCCF9093C60008952F9A80914E
:10133000C00087FFFCCF8091C60008958091C00057
:1013400087FD02C080E008958091C6000895EF9265
:10135000FF920F931F93DF93CF93CDB7DEB7C055A6
:10136000D0400FB6F894DEBF0FBECDBFFE01E75AE6
:10137000FF4F619171918E010F5F1F4FC801AF0147
:1013800008DF7C0103C0C9DF0F5F1F4FF8018081B8
:101390008823C9F7C701C05BDF4F0FB6F894DEBFE3
:1013A0000FBECDBFCF91DF911F910F91FF90EF90B6
:1013B00008955058BB27AA270ED075C166D130F0CA
:1013C0006BD120F031F49F3F11F41EF45BC10EF499
:1013D000E095E7FB51C1E92F77D180F3BA17620797
:1013E00073078407950718F071F49EF58FC10EF40A
:1013F000E0950B2EBA2FA02D0B01B90190010C0125
:10140000CA01A0011124FF27591B99F0593F50F43C
:10141000503E68F11A16F040A22F232F342F442794
:10142000585FF3CF469537952795A795F04053958C
:10143000C9F77EF41F16BA0B620B730B840BBAF05C
:101440009150A1F0FF0FBB1F661F771F881FC2F7C7
:101450000EC0BA0F621F731F841F48F487957795DB
:101460006795B795F7959E3F08F0B3CF9395880F92
:1014700008F09927EE0F979587950895D9D008F42D
:1014800081E008950CD00FC107D140F0FED030F0BC
:1014900021F45F3F19F0F0C0511139C1F3C014D1EC
:1014A00098F39923C9F35523B1F3951B550BBB272B
:1014B000AA2762177307840738F09F5F5F4F220FD8
:1014C000331F441FAA1FA9F333D00E2E3AF0E0E8D1
:1014D00030D091505040E695001CCAF729D0FE2F1D
:1014E00027D0660F771F881FBB1F261737074807AF
:1014F000AB07B0E809F0BB0B802DBF01FF27935865
:101500005F4F2AF09E3F510568F0B6C000C15F3FB3
:10151000ECF3983EDCF3869577956795B795F7954C
:101520009F5FC9F7880F911D9695879597F9089544
:10153000E1E0660F771F881FBB1F621773078407E0
:10154000BA0720F0621B730B840BBA0BEE1F88F7EF
:10155000E095089504D06894B111D9C00895BCD025
:1015600088F09F5790F0B92F9927B751A0F0D1F08C
:10157000660F771F881F991F1AF0BA95C9F712C016
:10158000B13081F0C3D0B1E00895C0C0672F782F8B
:101590008827B85F39F0B93FCCF386957795679582
:1015A000B395D9F73EF490958095709561957F4FEE
:1015B0008F4F9F4F0895E89409C097FB3EF4909594
:1015C0008095709561957F4F8F4F9F4F9923A9F01C
:1015D000F92F96E9BB279395F695879577956795AB
:1015E000B795F111F8CFFAF4BB0F11F460FF1BC0EF
:1015F0006F5F7F4F8F4F9F4F16C0882311F096E982
:1016000011C0772321F09EE8872F762F05C066232F
:1016100071F096E8862F70E060E02AF09A95660FE8
:10162000771F881FDAF7880F9695879597F90895A1
:10163000990F0008550FAA0BE0E8FEEF16161706E3
:10164000E807F907C0F012161306E407F50798F04B
:10165000621B730B840B950B39F40A2661F0232B64
:10166000242B252B21F408950A2609F4A140A695E0
:101670008FEF811D811D089597F99F6780E870E0C5
:1016800060E008959FEF80EC089500240A941616F8
:10169000170618060906089500240A941216130660
:1016A000140605060895092E0394000C11F48823EE
:1016B00052F0BB0F40F4BF2B11F460FF04C06F5F0A
:1016C0007F4F8F4F9F4F089557FD9058440F551FE0
:1016D00059F05F3F71F04795880F97FB991F61F0B4
:1016E0009F3F79F087950895121613061406551F2B
:1016F000F2CF4695F1DF08C0161617061806991F97
:10170000F1CF86957105610508940895E894BB278B
:1017100066277727CB0197F908950BD0C4CFB5DFA3
:1017200028F0BADF18F0952309F0A6CFABCF11242B
:10173000EECFCADFA0F3959FD1F3950F50E0551F70
:10174000629FF001729FBB27F00DB11D639FAA2716
:10175000F00DB11DAA1F649F6627B00DA11D661F65
:10176000829F2227B00DA11D621F739FB00DA11D86
:10177000621F839FA00D611D221F749F3327A00D40
:10178000611D231F849F600D211D822F762F6A2FDC
:1017900011249F5750408AF0E1F088234AF0EE0F61
:1017A000FF1FBB1F661F771F881F91505040A9F76E
:1017B0009E3F510570F060CFAACF5F3FECF3983E9B
:1017C000DCF3869577956795B795F795E7959F5FD5
:1017D000C1F7FE2B880F911D9695879597F908956F
:1017E00011F40EF44FCF3EC077DFD0F39923D9F335
:1017F000CEF39F57550B87FF43D00024A0E640EA65
:10180000900180585695979528F4805C660F771F55
:10181000881F20F026173707480730F4621B730B28
:10182000840B202931294A2BA6951794079420254B
:1018300031254A2758F7660F771F881F20F0261793
:101840003707480730F4620B730B840B200D311DF2
:10185000411DA09581F7B901842F9158880F969565
:10186000879508959F3F31F0915020F487957795A3
:101870006795B795880F911D9695879597F9089567
:1018800091505040660F771F881FD2F70895629FCE
:10189000D001739FF001829FE00DF11D649FE00D68
:1018A000F11D929FF00D839FF00D749FF00D659FC9
:1018B000F00D9927729FB00DE11DF91F639FB00DC8
:1018C000E11DF91FBD01CF0111240895AA1BBB1B07
:1018D00051E107C0AA1FBB1FA617B70710F0A61B30
:1018E000B70B881F991F5A95A9F780959095BC0151
:1018F000CD01089597FB092E07260AD077FD04D065
:10190000E5DF06D000201AF4709561957F4F0895A9
:10191000F6F7909581959F4F0895A1E21A2EAA1B84
:10192000BB1BFD010DC0AA1FBB1FEE1FFF1FA2178F
:10193000B307E407F50720F0A21BB30BE40BF50B8C
:10194000661F771F881F991F1A9469F76095709515
:10195000809590959B01AC01BD01CF010895FC01DC
:1019600088279927E89421912032E9F3293010F053
:101970002E30C8F32B3239F02D3231F4689403C085
:101980000BD0820F911D219120532A30C8F31EF4F1
:10199000909581959F4F08957AE0979F902D879F0E
:0C19A000802D910D11240895F894FFCFC4
:1019AC0068656C6C6F000D0A232068656C6C6F0D9C
:1019BC000A00232064656C61792025690D0A006496
:1019CC00656C617920256900232074696D656F75DC
:1019DC00742025690D0A0074696D656F7574202576
:1019EC0069002320417667732025690D0A00417632
:1019FC0067732025690023204441432025690D0A83
:101A0C0000442025690025692000256620256620D4
:101A1C00002569000D0A00706F6C6C00256C2000AD
:0A1A2C000D0A003F003F0D0A000301
:00000001FF
